:020000040000FA
:0600000000308600072815
:08000800AD0A0B1109000313FE
:1000100083121030850007309900A0308B0000302B
:1000200083168C00C53081000030860004308500C6
:100030008312203084008001840A041F1B280030B2
:10004000AB0014222130D023AE002430D023B100E5
:100050002230D023B800B3000230D023BE001E30BF
:10006000D023C0002330D023AC00AC182C150430B2
:10007000B5003C128512E421C2208D20FB202222F3
:100080003C28043005052A060319B90A08002A1D70
:100090004C28051D4928080005194C2808002A1974
:1000A0004C284928AD017120043005052A060319A2
:1000B0005C28AD186A285328712071207120B9017D
:1000C00041207120712041207120DD20412002302B
:1000D000390208002030C2002F08C100BA2347208F
:1000E00022282B1880288510010C7F3903197C28C1
:1000F0002F02031C85100800AF08031D851408009B
:100100008510010C7F39031989282F02031C8510E3
:100110000800AF08031D851408002508A100260863
:10012000A2002708A3002808A400A501A601A70192
:10013000A801253084009F20A720AF2008000830A8
:10014000A9004F205220800DA90BA1280800840A85
:100150004F205220800D4F205220800D0800840A2D
:100160000430A9004F205220800C840A4F205220D6
:10017000800CA9030319BE288403B228800E8403CF
:10018000800E08002030B9001330A90004300505A6
:100190002A060319D028B90BD3280430AA06C2288E
:1001A0002A30A900CB28043005052A060319C428E3
:1001B0007120DD20A90BD3280800BC1CF8283208C8
:1001C0002F02031CF62803103B0D2C1C3B08323E6B
:1001D0002C180A3EA000010CA002031808007D3C68
:1001E000031CF42886100800861408008614712861
:1001F000AC188610712821082502031D1B2922082E
:100200002602031D1B2923082702031D1B2924087E
:100210002802031D1B2921082E02031915292C1F52
:100220001B2921083102031D1B29712023082402E8
:100230000319A8291C2908003C162808FE3E0319AA
:100240004329FF3E03198510FF3E03198610FF3E28
:1002500003194929FF3E03199421FF3E031979210F
:10026000FD3E03194E29FF3E03198514FF3E031975
:100270008614FF3E03194629FF3E03199E21FF3EC7
:1002800003198721C2292308073C6D292308F83E5A
:100290006D292308073C031861296D2908302702BE
:1002A000031C6D2903191B29FD3E03198514FF3E0C
:1002B00003198614FE3E03199E21FF3E0319872170
:1002C000C22903197921FF3E03199421FE3E031927
:1002D0008610FF3E03198510C229240801392B0618
:1002E0000319C22924080139AB001C220130A300E4
:1002F000C229AC1E8529BC1E0800B9002230D023BB
:10030000B800B300BC123908080085110800AC1E03
:100310009229BC1A0800B9000130B800B300BC161D
:1003200039080800851508002C1D9C29AC1C9A2949
:10033000BC1008003C110800851208002C1DA629DD
:10034000AC1CA429BC1408003C1508008516080044
:1003500071202308013A031DBD293C18B329FF3041
:10036000B4000430B5003C1866223C18C2293C1485
:10037000AB090130AB051C22C229AC18BC143C1CD3
:10038000C2293C107120E4212308013A0319E12914
:100390002308BB003C19D9290310BB0DAC1FDD2974
:1003A000A2080319DD29221CBB0AA218DD29BB0AF9
:1003B000DD293C1EDD293030BB073B08D023B200CD
:1003C0000800B201AF0108002C1A062A2B18F729E1
:1003D00005100516AF0803190512AC1D05163C1AC9
:1003E0000800A218F52986100800861408000512D6
:1003F0000514AF0803190510AC1D05143C1A0800BC
:10040000A218042A86100800861408002B180E2A49
:100410000510A2180516A21C051208000512A21844
:100420000514A21C051008002030D023AF00B20034
:100430002530D023AB0008002530C2002B08C100B6
:10044000BA2308003808013C031D292A3208AF00EE
:1004500008003C1232082F0203190800B30B0800F1
:100460003E082F0203183D2AB20803193A2A3E0813
:10047000AF003D2AAF01B30A080032082F02031C67
:10048000432AAF03442AAF0A3808B300AD0126302F
:10049000D0232F08BF00C10B4E2A522ABF070318D2
:1004A000AD0A4B2A0430C100AD0CBF0CAD13C10B1B
:1004B000542AAD0803185E2AAD0CBF0C2730D02398
:1004C0003F084102031C0030B3070800B40B0800CA
:1004D0006A2A0800FF30B400B50B0800A02AB60055
:1004E000B60A0B30BC1BD62BB60B772A08000516B4
:1004F0000514D62305120510D623742A0230B6003F
:100500002F30722A8D222308013A0319822A8D2264
:100510002308013A031D872A0800C2208D202108E4
:100520002502031D8D2A22082602031D8D2A230879
:100530002702031D8D2A24082802031D8D2A080086
:10054000BC1009306F2201306F228222DC23B903F4
:100550000319D12AB9030319D92AB9030319E42AC3
:10056000B90303191E2BB9030319342BB90303195B
:10057000462BB90303194E2BB9030319602BB9039A
:100580000319732BB9030319852BB9030319982B8E
:100590000430B9020319A62B21080319B22B7E22BD
:1005A000A52A6F2282222130C2002108C100BA236D
:1005B000A32A6F2282222230C200DC233908C10024
:1005C0002230C200BA23A32A6F228222DC23C20077
:1005D0000310C20D21080319032B10303902031C2C
:1005E000F32A7E22E52A39086F228222DC230310B7
:1005F000B90DB91FFD2A7E22F52A3908C100BA2398
:1006000001306F22E52A0630B600D023B900B603C8
:100610003603D023B9020310390CC1073608C200D3
:10062000BA2383169C18122B8312B60A1E30360288
:100630000318A32AB60AB60A3608052B6F228222AF
:10064000DC2304303902031C272B7E221F2B23308E
:10065000D023E730C105B9033918C115B9184116BF
:100660002330C200BA23A32A6F228222DC23033064
:100670003902031C3D2B7E22352B2330D023C1129F
:10068000391CC1162330C200BA23A32A6F2282224A
:100690002430C2002108C100BA23A32A6F2282227B
:1006A000DC2303303902031C572B7E224F2B2330CF
:1006B000D0234113391C41172330C200BA23A32A87
:1006C0006F228222DC2305303902031C692B7E2233
:1006D000612B2330D023F830C1053908C104233001
:1006E000C200BA23A32A6F228222DC2303303902FC
:1006F000031C7C2B7E22742B2330D023C113391C86
:10070000C1172330C200BA23A32A6F228222DC231E
:1007100004303902031C902B21303902031C922B28
:100720007E22862B2630C2003908C100BA23A32AB4
:100730006F228222DC23B908031DA02B7E22992B75
:100740002730C2003908C100BA23A32A8222DC2341
:1007500003303902031CAE2B7E22A62BBC13391C9E
:10076000BC17A32AFF30B4000430B50001306F225B
:100770008C212228410883169A008312420883168E
:100780009B008B131C129C111C1555309D00AA3028
:100790009D009C141C119C18CB2B83128B170800F6
:1007A00083169B001C141A0883120800AD01AD02C9
:1007B000AD08031DD82B0800B901A11FE22BB90A0F
:1007C000211FB90AA11EE82B0330B907211EB90762
:1007D000A11DEE2B0930B907211DB907A11CF42B6F
:0C07E0001B30B907211CB90739080800BC
:02400E00C401EB
:104200000000000012000000140015001600180045
:104210001A001C001E0020002200250028002B0090
:104220002E00320036003A003E00430048004E00A7
:1042300054005A00600067006E0075007C000000AA
:1042400000002A00030020002A00000010001E00C9
:10425000000000000000000000000000000000005E
:104260000000000008000A000C000E001000120000
:10427000150018001B001E002100250029002D003C
:10428000FF00FF00FF00FF00FF00FF00FF00FF0036
:10429000FF00FF00FF00FF00FF00FF00FF00FF0026
:1042A000FF00FF00FF00FF00FF00FF00FF00FF0016
:1042B000FF00FF00FF00FF00FF00FF00FF00FF0006
:1042C000FF00FF00FF00FF00FF00FF00FF00FF00F6
:1042D000FF00FF00FF00FF00FF00FF00FF00FF00E6
:1042E000FF00FF00FF00FF00FF00FF00FF00FF00D6
:1042F000FF00FF00FF00FF00FF00FF00FF00FF00C6
:00000001FF
